:020000040000FA
:10000000803102288731FD2F8331CE2B8331E42BC1
:100010008331D22B8331D62B8331DA2B8331E02B02
:1001540024001614161C0800AC2824001615161DBD
:100164000800B128FE0012001E00FE0BB528003462
:1001740080302400940028309500970109309200C3
:100184000800FA007830F9007908F000F101F10A6A
:100194007A08823131220800F7007708F5007508E3
:1001A400F000F101F10A76308131B52176080800BA
:1001B400F000200091117008240091002000911D8E
:1001C400E0282400160808002000A2007C30A000CB
:1001D4002008F0000230A1002108F1002208823139
:1001E400312208008031AA20803152308031DA2057
:1001F4008031C0308031DA2080318031AF20080076
:10020400F9007908F7007708F0000230F800780860
:10021400F1007A308131B5217B08F6007A08F500C7
:1002240008008031AA20813152308031DA208131B6
:1002340086308031DA20813110308031DA2081310A
:100244008031AF2008008031AA20813152308031C2
:10025400DA20813186308031DA20813111308031E9
:10026400DA2081318031AF200800F1002400961596
:10027400141C3A291108F0007008F200710C031CD8
:100284009612031896161616161A462972080800AE
:100294008031AA20813152308031DA20813180309E
:1002A4008031DA20813100308031DA2081318031AF
:1002B400AF202700161208008031AA208131523065
:1002C4008031DA208131A4308031DA208131710823
:1002D4008031DA20813172088031DA208131803135
:1002E400AF20080022008C128E100C128E120C11FA
:1002F4000E100C1027001512981500308231682258
:100304008131013A031D7F2922008E148431C924CE
:1003140081310230FB007B08F8000A308031C320B1
:10032400080022008E148C120C128E120C110E1066
:100334000C10270015129815013082316822813182
:10034400FB007B08FC007C08031DB0290330FB0084
:100354007B08F8000A308031C3200800F8010A3015
:100364008031C3200800F4007408F2007208F3001E
:1003740031009518BA291517700891007030920051
:100384000130F102710A0319080015141308F20070
:10039400730886008701720881000130F200720838
:1003A400F3070130F20072089107C2298031AA20B4
:1003B400813152308031DA20813180308031DA204D
:1003C400813103308031DA2081318031AF208131B5
:1003D4008031AA20813152308031DA20813181305C
:1003E4008031DA20813112308031DA20813180315C
:1003F400AF2081318131132108008031AA2081315D
:1004040052308031DA208131AC308031DA208131D0
:100414008031AA20813153308031DA20813100309B
:10042400813137218131F500F6017508F80076082D
:10043400F9000130813137218131F500F601750869
:10044400F600F50178087504F80079087604F900D7
:100454008031AF207908F4007808F3000800F40034
:100464007008F2007208F30031009518362A151747
:100474007408FF3E91007030920094010130F10243
:10048400710A0319080031009518452A730886007B
:100494008701010893000130F2007208F30701306C
:1004A400F20072089107200003108B1B0314310023
:1004B400151555309600AA30960095149518602AA3
:1004C40015112000031C402A8B17402AF10020003C
:1004D4008E196E2A6400692A8230F000DE30890B9E
:1004E400712AF00B712A71080319802A21009016D1
:1004F40020009717FE3096003930950020009012A6
:100504002700991120008E19892A6400842A630027
:10051400000071080319972A2000901E972A2100D1
:1005240090122000971302300800F201C8307202C2
:100534000318AF2A20008E19AF2A0D30F000FC30CA
:10054400890BA22AF00BA22A64000130F000700883
:10055400F207C8307202031C9C2A20009713C8308B
:100564007206031DB72A013008000030080022007B
:100574008C128E100C168E120C110E100C10210001
:100584009016270098151512991116122000971726
:10059400CA309600C9309500901227009911630063
:1005A40000002000901EEA2A0830813102218231A5
:1005B4007508013EFC000030763DFD0008308031B6
:1005C400E6208231CA3020009600C930950090128E
:1005D4002700991DD12A2000B301B40120008E19EF
:1005E400042B07303402D130031933020318042BCF
:1005F4000130B3070030B43DC8300032890BFF2A04
:100604006400F02A07303402D0300319330203188F
:100614003E2B9713B101B20108308131022182319E
:10062400760820003202031D192B750831020318C5
:100634003C2B22000C1582302000AF00DD30890BEA
:10064400212BAF0B212B003222000C110330200090
:10065400B0008A30AF005530890B2E2BAF0B2E2BF8
:10066400B00B2E2B0032640001302000B1070030A3
:10067400B23D0E2B9717CF2A97130230AF002F08E5
:10068400FB0001308631D226080023008C018D0145
:1006940004308E0022008C018D018E01D83024009C
:1006A4008E0090308D0021008C01F0308D00DC3004
:1006B4008E0018303D009D000D303C00A000193024
:1006C4003D009E000E303C00A10022008C10FF3043
:1006D40032009100FF309200FF309300FF3094000D
:1006E400FF309500FF3096001111111011131210F4
:1006F400931295106030990003309F00210010166A
:100704000B1720009713171618081F398038980004
:1007140018161808F0390B3898008031BA20833144
:100724000D302000B500FB30890B962BB50B962BB2
:1007340000322000031AB62B22000C158230200050
:10074400B500DD30890BA42BB50BA42B003222009D
:100754000C1182302000B500DD30890BAF2BB50BB6
:10076400AF2B003264009E2B0A308031CE208331BF
:10077400003A0319C42B0A308031CE208331023A67
:10078400031DE72B20008E19E72BFB01FB0A003029
:100794008631D2268331E72B813174218331E72BD3
:1007A400813193218331E72B8331FF238331E72B7D
:1007B40002302000B5003508FB00C92B8231B92274
:1007C4008331E72B8531B225833164000A308031CF
:1007D400CE2083312000B500B6013608003A031953
:1007E400F42BE72B35088400063004020318E72BAA
:1007F40080310435043E8200E72B22008C168E14CF
:100804000C128E120C110E100C10270015169811D4
:100814000030FC00FD0008308031E62083312000E8
:10082400A701A8014E30280220300319270203181B
:10083400362C8E19252C0230A3002308F8000A3028
:100844008031C3200800C8300032890B262C640094
:1008540001302000A7070030A83D4E302802203088
:1008640003192702031C1B2C8131D821833120005A
:10087400A701A80100302802053003192702031834
:10088400562C8031F420833120000D1E4B2C640043
:10089400462C0130A7070030A83D0030280205305F
:1008A40003192702031C432C813125218331813113
:1008B400FF21833174082000A6007308A500FF30CF
:1008C4002602EC3003192502031C6C2CEA30A50027
:1008D400FF30A6002508143EF1000030263DF2004A
:1008E40081315E21833122008E1005302000A30067
:1008F4002308F8000A308031C320833164000630B5
:100904002000A4001330A300AD30890B872CA30B67
:10091400872CA40B872C0032640006302000A4002E
:100924001330A300AD30890B952CA30B952CA40B8D
:10093400952C0032640022008C1227009911640067
:100944008031F42083312700161220000D1EA72CBD
:10095400630000008131FF21833174082000A60068
:100964007308A50000302602143003192502031C65
:10097400A12C81314A21833104302000A3002308B3
:10098400F8000A308031C32022008C1608002200AF
:100994000C148E148E160E1464000630F1001330FD
:1009A400F000AE30890BD42CF00BD42CF10BD42CEA
:1009B4006400493021009D00C3309E008230220033
:1009C4009700C8300032890BE42C21009D149D1837
:1009D400E92C22008C128E100C128E120C110E10A7
:1009E4000C1021001D102200971321001C08F00098
:1009F400F1017008F9007108FA001B08F000F10118
:100A04007908F300F20170087204F40071087304A9
:100A1400F5007408F9007508FA0003307A022E30E4
:100A2400031979020318322D03307A0215300319A1
:100A340079020318322D02307A02FC30031979024C
:100A44000318322D02307A02E330031979020318B5
:100A5400322D02307A02CA3003197902031C342D74
:100A64000630572D02307A02B13003197902031C83
:100A74003D2D0530572D02307A0298300319790242
:100A8400031C462D0430572D02307A027F3003199F
:100A94007902031C4F2D0330572D02307A02663041
:100AA40003197902031C5B2D0230F0007008F80072
:100AB400662D02307A024D3003197902031C652D2C
:100AC400F801F80A662DF801F601F7010130770202
:100AD400F430031976020318080078080319742DFA
:100AE40022008E14C8300032890B752D22008E101E
:100AF4000230780203188C16C8300032890B7F2D1F
:100B040022008C120330780203188E16C83000328B
:100B1400890B892D22008E120430780203180C16DA
:100B2400C8300032890B932D22000C120530780254
:100B340003180E14C8300032890B9D2D22000E10AC
:100B44000630780203180C15C8300032890BA72D23
:100B540022000C1164000130F6070030F73D682DC7
:100B64002000B10122008C128E140C168E160C116A
:100B74000E100C102700151298152000B201B301B5
:100B84004E3033022030031932020318432E0E1A5A
:100B9400DE2D3108203E860087018101810A013063
:100BA400FB007B08B1070E1ED52D8230FB00DE3022
:100BB400890BDA2DFB0BDA2D20008E1BF62D02306B
:100BC400FB003108203E860087017B08810001304C
:100BD400FB007B08B1078E1FED2D8230FB00DE3059
:100BE400890BF22DFB0BF22D20008D1B0E2E0330F2
:100BF400FB003108203E860087017B08810001301C
:100C0400FB007B08B1078D1F052E8230FB00DE3010
:100C1400890B0A2EFB0B0A2E20000E1B262E0430F5
:100C2400FB003108203E860087017B0881000130EB
:100C3400FB007B08B1070E1F1D2E8230FB00DE3047
:100C4400890B222EFB0B222E083020003106031DB7
:100C54002D2E22000E141030200031020318432ED2
:100C64006400C8300032890B342E01302000B207F2
:100C74000030B33D4E303302203003193202031CDE
:100C8400C92D203032064E3003193306031D522E6F
:100C94000230FB007B08F8000A308031C3200800D2
:100CA400B001B00AB201B3010030330208300319B5
:100CB40032020318772E3208083E203E8600870150
:100CC4003208203E840085010008010603196C2EB9
:100CD400B001772E0130B2070030B33D003033024B
:100CE400083003193202031C5D2E3003031DCA2E83
:100CF40022000C128E108E120E108230FB00DE3099
:100D0400890B822EFB0B822E22008E148E160E145B
:100D14008230FB00DE30890B8D2EFB0B8D2E2200E2
:100D24008E108E120E108230FB00DE30890B982E4E
:100D3400FB0B982E22008E148E160E148230FB00AC
:100D4400DE30890BA32EFB0BA32E2000B201B301CE
:100D5400003033020830031932020318CA2E320855
:100D6400203E860087010108FB007B08F80032085A
:100D7400003E8031C320853101302000B2070030AD
:100D8400B33D00303302083003193202031CB12E84
:100D94000230FB007B08F8000A308031C3200800D1
:100DA4002000AA00AE012A08031DDF2E7B030319CD
:100DB400DF2E22008C168E10F32E2A080319F02E33
:100DC4007B030319F02E22008C128E100C128E1647
:100DD4000C110E102000A901A90AFC2E22008C126D
:100DE4008E140C128E160C110E100330FC007C08AD
:100DF4002000A90022000C102700151298110B30B6
:100E04008031CE208631FC00200029087C020318A2
:100E1400F02F2000AB01AC0175302C0230300319E7
:100E24002B020318A32F0E1A2A2F2E08203E860009
:100E340087018101810A0130FC007C08AE070E1E87
:100E4400212F8230FC00DE30890B262FFC0B262F4D
:100E540020008E1B422F0230FC002E08203E86000C
:100E640087017C0881000130FC007C08AE078E1FDE
:100E7400392F8230FC00DE30890B3E2FFC0B3E2FD5
:100E840020008D1B5A2F0330FC002E08203E8600C4
:100E940087017C0881000130FC007C08AE078D1FAF
:100EA400512F8230FC00DE30890B562FFC0B562F5D
:100EB40020000E1B722F0430FC002E08203E8600FA
:100EC40087017C0881000130FC007C08AE070E1FFE
:100ED400692F8230FC00DE30890B6E2FFC0B6E2FE5
:100EE400083020002E02031C922FA801A80AAD018D
:100EF40008302D020318A32F2D08203E84008501FD
:100F04002D08003E8031CE208631000603198C2F37
:100F14002000A8010130FC007C082000AD077A2FD6
:100F2400C8300032890B932F640001302000AB07D6
:100F34000030AC3D75302C02303003192B02031CF9
:100F4400152F30302B06753003192C06031DB32FD3
:100F54000330FC007C08F8000B308031C32086315C
:100F6400012F20002803031DC42F7B08FC007C08EC
:100F7400F8000A308031C3208631F8010B3080310B
:100F8400C32008000B308031CE208631013EFC00A6
:100F94007C08F8000B308031C320863122000C1607
:100FA40064000630FD001330FC00AE30890BD82FEE
:100FB400FC0BD82FFD0BD82F64000630FD00133036
:100FC400FC00AE30890BE42FFC0BE42FFD0BE42F67
:100FD400640022000C122000AE01012F0530FC0039
:100FE4007C08F8000A308031C3208631F8010B30C8
:0C0FF4008031C320080020008331472B0F
:020000040001F9
:08000E00ECFF1BFFFFDFFCFF0C
:10E000000100010001000100010001000100010008
:08E01000000000000000000008
:00000001FF
